:100000000C94E7000C9478120C9451120C940F018C
:100010000C940F010C940F010C940F010C940F0120
:100020000C940F010C940F010C940F010C94AF145D
:100030000C940F010C94BE130C940F010C940F013F
:100040000C940F120C940F010C94DD110C94B71149
:100050000C940F010C940F010C940F010C940F01E0
:100060000C949F120C940F0197A0895B5A0F830D7B
:10007000C95F6035C2E907E18C24671E458E0863BD
:1000800025F0150A17BE0694F778EA4B001AC53E0C
:100090005EFCDBCB75230B2039B12158ED95385729
:1000A000AE147D88ABA844AF4AA547868B301BA60B
:1000B0004D929EE7536FE57A3CD385E6DC695C2977
:1000C000372EF528F4668F3641193FA101D85049E3
:1000D000D14C84BBD05912A9C8C4878274BC9F5626
:1000E000A4646DC6ADBA034034D9E2FA7C7B05CA7C
:1000F0002693767EFF5255D4CFCE3BE32F103A1194
:10010000B6BD1C2ADFB7AAD577F898022C9AA34669
:10011000DD99659BA72BAC09811627FD13626C6ED8
:100120004F71E0E8B2B97068DAF661E4FB22F2C11F
:10013000EED2900CBFB3A2F1513391EBF90EEF6BFD
:1001400031C0D61FB5C76A9DB854CCB07379322D73
:100150007F0496FE8AECCD5DDE72431D1848F38D58
:1001600080C34E42D73D9CB4970000000024002776
:10017000002A0000000000250028002B00000000DD
:1001800000230026002900040404040404040402DB
:100190000202020202030303030303020203010239
:1001A0000408102040800102040810200102040805
:1001B00010204080400000000900030200000405F8
:1001C000080000000000000000000000EC141124F2
:1001D0001FBECFEFD8E0DEBFCDBF11E0A0E0B1E0A1
:1001E000E2EAF5E502C005900D92AE39B107D9F704
:1001F00024E0AEE9B1E001C01D92A030B207E1F702
:1002000010E0C7EED0E004C02197FE010E94A92AA9
:10021000C63ED107C9F70E9481150C94CF2A0C94D1
:10022000000008950895982F2091CA0381E021329B
:1002300008F043C08091C9038111FCCF809118035D
:1002400032E03093C9039093C8039FEF9093F60276
:100250001092F5022093F402A8EFB2E0E4EDF2E090
:1002600090E0291331C01092D3029091D302880FED
:10027000892B8093D3028091C703813049F5109276
:10028000C7038091D3028093BB008091BC0083FDA3
:10029000F8CF85EC8093BC008091C9038230E1F3F4
:1002A0008091F6028F3FB1F08091F6028032A1F08A
:1002B0008091F602803391F084E01092CB0310928B
:1002C000CA031092F70208953D9131939F5FC9CF01
:1002D00085EEE0CF80E0F1CF82E0EFCF83E0EDCF9D
:1002E0008091CC039091CD03891B990B089580E9EF
:1002F00091E00895AF92BF92CF92DF92EF92FF927A
:100300000F931F93CF93DF936C017B018B01040F3D
:10031000151FEB015E01AE18BF08C017D10759F0D9
:100320006991D601ED91FC910190F081E02DC6011B
:100330000995892B79F7C501DF91CF911F910F9115
:10034000FF90EF90DF90CF90BF90AF900895FC01A9
:10035000538D448D252F30E0842F90E0821B930B2A
:10036000541710F0CF96089501970895FC01918DD0
:10037000828D981761F0A28DAE0FBF2FB11D5D96D3
:100380008C91928D9F5F9F73928F90E008958FEF75
:100390009FEF0895FC01918D828D981731F0828D29
:1003A000E80FF11D858D90E008958FEF9FEF089580
:1003B000FC01918D228D892F90E0805C9F4F821BE4
:1003C00091098F739927089589E193E00E94D801DC
:1003D00021E0892B09F420E0822F089580E090E04D
:1003E000892B29F00E94E40181110C9400000895EA
:1003F000FC01A48DA80FB92FB11DA35ABF4F2C919A
:10040000848D90E001968F739927848FA689B78990
:100410002C93A089B1898C9180648C93938D848D69
:10042000981306C00288F389E02D80818F7D808338
:100430000895EF92FF920F931F93CF93DF93EC01F8
:1004400081E0888F9B8D8C8D981316C0E889F9897F
:10045000808185FF11C0EE89FF896083E889F98971
:1004600080818064808381E090E0DF91CF911F9153
:100470000F91FF90EF900895F62E0B8D10E00F5F17
:100480001F4F0F731127E02E8C8D8E110CC00FB6ED
:1004900007FCFACFE889F989808185FFF5CFCE0185
:1004A0000E94F801F1CFEB8DEC0FFD2FF11DE35A07
:1004B000FF4FF0820B8FEA89FB8980818062D2CF67
:1004C000CF93DF93EC01888D8823B9F0AA89BB898B
:1004D000E889F9898C9185FD03C0808186FD0DC076
:1004E0000FB607FCF7CF8C9185FFF2CF808185FF97
:1004F000EDCFCE010E94F801E9CFDF91CF910895B1
:10050000843081F028F48230E9F08330F9F00895E6
:10051000883071F0893091F08530B9F48091800095
:100520008F7D03C0809180008F7780938000089535
:100530008091B0008F778093B00008958091B000D3
:100540008F7DF9CF84B58F7784BD089584B58F7D75
:10055000FBCFCF93DF93282F30E0F901EB54FE4F10
:100560008491F901E256FE4FD491F901E957FE4F0B
:10057000C491CC23A1F081110E948002EC2FF0E005
:10058000EE0FFF1FE358FE4FA591B491EC91ED23C0
:1005900081E090E009F480E0DF91CF91089580E060
:1005A00090E0FACF1F93CF93DF93282F30E0F9012B
:1005B000EB54FE4F8491F901E256FE4FD491F901BC
:1005C000E957FE4FC491CC23A9F0162F81110E9448
:1005D0008002EC2FF0E0EE0FFF1FED58FE4FA591CB
:1005E000B4918FB7F894EC91111108C0D095DE2327
:1005F000DC938FBFDF91CF911F910895DE2BF8CF51
:10060000CF93DF9390E0FC01E256FE4F249189578F
:100610009E4FFC0184918823C9F090E0880F991FB8
:10062000FC01E759FE4FA591B491FC01ED58FE4F36
:10063000C591D49161110DC09FB7F8948C9120950C
:1006400082238C938881282328839FBFDF91CF91B9
:100650000895623051F49FB7F8943C91822F8095B1
:1006600083238C93E8812E2BEFCF8FB7F894EC91F6
:100670002E2B2C938FBFEACF883020F08D3008F4DA
:100680008DE08E508770806480937C0080917A002A
:10069000806480937A0080917A0086FDFCCF8091FF
:1006A0007800909179000895CF92DF92EF92FF92B7
:1006B0006FB7F8948091EA019091EB01A091EC0161
:1006C000B091ED015091E90126B535B3432F41704A
:1006D00030FF04C041E02F3F09F440E06FBF6C01E0
:1006E0007D0137E0CC0CDD1CEE1CFF1C3A95D1F7E8
:1006F000C50ED11CE11CF11CC81AD90AEA0AFB0A72
:10070000880F991FAA1FBB1FC81AD90AEA0AFB0A39
:1007100063E0CC0CDD1CEE1CFF1C6A95D1F730E0C9
:10072000A3E3B3E00E946A2A672F782F892F9927C5
:100730006C0D7D1D8E1D9F1D442321F06D5C7C4F33
:100740008F4F9F4FFF90EF90DF90CF9008958F9243
:100750009F92AF92BF92CF92DF92EF92FF926B0186
:100760007C010E9454034B015C01C114D104E104DB
:10077000F104B9F00E945403681979098A099B09A8
:10078000683E73408105910580F321E0C21AD108CB
:10079000E108F10888EE880E83E0981EA11CB11CC8
:1007A000E4CFFF90EF90DF90CF90BF90AF909F90FD
:1007B0008F9008952FB7F8946091EA017091EB0142
:1007C0008091EC019091ED012FBF08950F931F933D
:1007D0008091DA039091DB03DC01ED91FC910084C0
:1007E000F185E02D0995892B09F4D7C060E070E010
:1007F000CB010E94A7032091F8038091DA03909126
:10080000DB03DC01ED91FC910284F385E02D2111E5
:100810000BC009958093E4038E37D1F68091F803DD
:100820008F5F8093F803D4CF09959091F803E92F57
:10083000F0E0E652FC4F82879230B9F09930D9F05F
:100840009130A9F48F3F99F01092F80381E08093E2
:10085000FA031092FD031092FC038093FE031092A2
:10086000FF0380E01F910F910895863069F79F5F25
:100870009093F803ADCF8F3E39F72091E603809136
:10088000E503280F3327331FE091E703C9018E0FDB
:10089000911D2091E803280F392F311D4091E90364
:1008A00050E0240F351F8091EA0390E06091EB0344
:1008B00070E0762F6627F091EC036F0F711D280F03
:1008C000391F3195219531096217730709F0BCCFA3
:1008D0001092F803E13419F41092FF032FC0E09353
:1008E000FB03542F4427840F951F9093FD0380939F
:1008F000FC03EA53E63108F046C0F0E0EE57FB4F48
:100900000C94A92AAF04B704C1049804C104A1043B
:10091000BF04C304C104C104C104C104C104C104AF
:10092000C104C104C304C104C104C104C104C1049D
:1009300085E08093FA0381E08093FE038091FE03BB
:1009400091CF80FF02C089E0F4CF81FF02C084E034
:10095000F0CF83709927892B89F38AE0EACF80FF53
:1009600002C087E0E6CF81FFE9CF82E0E2CF80FFDF
:1009700002C088E0DECF81FFE1CF83E0DACF86E0FE
:10098000D8CF8BE0D6CF81E08093FA031092FD039D
:100990001092FC038093FE039FCF8091FF03882376
:1009A00069F20E94DA030091DC031091DD032091CB
:1009B000DE033091DF03601B710B820B930B009100
:1009C000E0031091E1032091E2033091E30360170B
:1009D00071078207930708F4B1CF1092F8031092C1
:1009E000FA031092FD031092FC0381E036CF80934E
:1009F000F103272F30E07093F3036093F4034091E9
:100A0000F0039091EF03490F5527551F840F952F41
:100A1000911D4091F203840F911D820F931F680F67
:100A2000792F711D7195619571097093F50360932C
:100A3000F603442361F08091FF03882341F060E0D6
:100A400070E0CB010E94A7030E94E603F4CF8091DF
:100A5000DA039091DB03DC01ED91FC910280F381DC
:100A6000E02D4AE050E06EEE73E009950E94DA0353
:100A70006093DC037093DD038093DE039093DF03C8
:100A80008091F20391E0811101C090E09093FF0307
:100A9000811106C06AE070E080E090E00C94A7034A
:100AA000089570E060E086E10C94F7044F925F9245
:100AB0006F927F929F92AF92BF92CF92DF92EF920E
:100AC000FF920F931F93CF93DF9300D01F92CDB768
:100AD000DEB7D090B6038091B9039091BA03A0918C
:100AE000BB03B091BC03892B8A2B8B2BD9F00E94BE
:100AF00054030091A8021091A9022091AA023091FA
:100B0000AB02601B710B820B930B0091B903109128
:100B1000BA032091BB033091BC03601771078207B1
:100B20009307C8F20E9454036093A8027093A9022D
:100B30008093AA029093AB02E091C103F091C203AB
:100B4000309759F04091BD035091BE036091BF03AF
:100B50007091C0038D2D0995D82EE090A602F090DB
:100B6000A7024D2C512C712C612CE114F10409F4D5
:100B700059C0D7011C96CC901C978091B7039091D7
:100B8000B8038436910510F41C961C92D701ED91A0
:100B9000FC91A280B38019821A821B82DD2079F138
:100BA000F701369610E000E02191222319F192809E
:100BB000992001F130E050E040E02F5F3F4F4F4F70
:100BC0005F4FC301B2010E94792A9B01AC01892DBC
:100BD00090E0B0E0A0E0BC01CD016F5F7F4F8F4F90
:100BE0009F4F0E94792AA1E0B0E0AC0FBD1FA00F7B
:100BF000B11F8C930F5F1F4F03301105A9F60981B8
:100C00001A812B81F7014585568562817381C70161
:100C1000F5010995D7011C96CC921C971496ED907E
:100C2000FC90A3CF8091A4029091A5028C010F5F4C
:100C30001F4F1093A5020093A4024997B4F10E949C
:100C4000DA03C090A002D090A102E090A202F0903E
:100C5000A3029B01AC012C193D094E095F0921F447
:100C600021E030E040E050E088EE93E0089FB001E2
:100C7000099F700D189F700D1124072E000C880B12
:100C8000990B0E94482A3093B8032093B70310921F
:100C9000A5021092A4020E94DA036093A00270934E
:100CA000A1028093A2029093A3020F900F900F9045
:100CB000DF91CF911F910F91FF90EF90DF90CF9038
:100CC000BF90AF909F907F906F905F904F900895EE
:100CD0008F929F92AF92BF92CF92DF92EF92FF924C
:100CE000CF936B017C010E94DA034B015C01C114BC
:100CF000D104E104F10441F4C090E003D090E10399
:100D0000E090E203F090E3030E94E603C82F811114
:100D100011C00E94DA03681979098A099B09C6166D
:100D2000D706E806F90630F060E070E0CB010E94DB
:100D3000A703EACF8C2FCF91FF90EF90DF90CF9059
:100D4000BF90AF909F908F90089570E060E082E434
:100D50000E94F70460E070E0CB010E9468068111F8
:100D600003C08FEF9FEF08951092FE038091FA0366
:100D70008B30B9F78091FC039091FD03089508959D
:100D800085ED8093BC008091BC0084FDFCCF109267
:100D9000C90308952091C501260F3327331F21323F
:100DA0003105ECF42091C903FC0190E080E024308F
:100DB00069F082E00895A091C5012191AC014B55E5
:100DC0005E4FA40FB52FB11D2C930196861798F393
:100DD0008091C501680F6093C50180E0089581E0AE
:100DE00008950895E091CD038091CC03E81730F485
:100DF000F0E0E455FD4F808190E008958FEF9FEF84
:100E000008959091CD038091CC032FEF3FEF981779
:100E100048F4E92FF0E0E455FD4F208130E09F5F7A
:100E20009093CD03C9010895CF92DF92EF92FF9284
:100E30000F931F93CF93DF937C01CB018A01209105
:100E4000F702222389F0EB016B01C40ED51ECC15ED
:100E5000DD0569F06991D701ED91FC910190F08178
:100E6000E02DC7010995F3CF642F0E94CA06C8017F
:100E7000DF91CF911F910F91FF90EF90DF90CF9076
:100E80000895CF93DF931F92CDB7DEB7698320918A
:100E9000F7022223F9F02091CA03203258F021E012
:100EA00030E0FC013383228390E080E00F90DF91FB
:100EB000CF9108958091CB03E82FF0E0E850FD4FEB
:100EC000998190838F5F8093CB038093CA0381E0E5
:100ED00090E0ECCF61E0CE0101960E94CA06F7CF08
:100EE000CF93DF93D1E0D093F70288E68093180385
:100EF0001092CB031092CA0360E08EEC93E00E9444
:100F0000410760E88EEC93E00E9441078091CD029A
:100F1000CAE06C2F0E94892A8295807F682F690F12
:100F20008EEC93E00E9441078091CE026C2F0E94CC
:100F3000892A8295807F682F690F8EEC93E00E944A
:100F400041078091CF026C2F0E94892A8295807F71
:100F5000682F690F8EEC93E00E9441078091D002C8
:100F60006C2F0E94892A8295807F682F690F8EECF2
:100F700093E00E9441078091D1026C2F0E94892A40
:100F80008295807F682F690F8EEC93E00E94410765
:100F90008091D2028E516C2F0E94892A8295807F87
:100FA000682F690F8EEC93E00E94410781E00E9458
:100FB000130181111DC0D093F7021092CB03109240
:100FC000CA0360E08EEC93E00E9441078091CC025E
:100FD0006C2F0E94892A8295807F682F690F8EEC82
:100FE00093E00E94410781E00E94130191E081118A
:100FF00090E0892FDF91CF91089590E080E00895EF
:10100000282F382F37FD2095229F020E20E0211D2A
:10101000000C221F37FD20951124822F0895BF92C6
:10102000CF92DF92EF92FF920F931F93CF93DF93B4
:10103000C62EE8E6F0E0E491E70F2E2F30E0F9014C
:10104000E859FF4FD490F901E759FF4FD491E9E6F1
:10105000F0E00491700F072F10E0F801E859FF4FFE
:10106000C49107591F4FF801E490182F1695F62EDA
:10107000F694BF2C0E940008082F8C2D0E940008B7
:1010800050E8510FEC2FF0E0E859FF4F2491452F25
:101090003F2D22FD02C04F2D352F20FD319521FD22
:1010A000419545953595341FED2DF0E0E859FF4FFA
:1010B000E491212FE2FF02C02F2DB12EE0FD2195FA
:1010C000E1FDB1944B2D45952595241F23170CF078
:1010D00051C0321B309F030E30E0311D1124320FFE
:1010E00040E84F0DEE2DF0E0E859FF4FE491242F3A
:1010F000E2FF02C0252F542FE0FD5195E1FD21951F
:1011000025955595521FED2FF0E0E859FF4FE491DA
:10111000E2FF03C0912F142F492FE0FD1195E1FD4F
:10112000419545951595141F15170CF02EC0511BB0
:10113000509F050E50E0511D1124912F950F391726
:101140000CF02DC0931B292F482F249F020E20E066
:10115000211D1124230F205C220F08F42FEF822F72
:10116000DF91CF911F910F91FF90EF90DF90CF9083
:10117000BF900895922F931B392F309F030E30E0BC
:10118000311D1124231B322FABCF212F251B209F74
:10119000020E20E0211D1124912F921BD0CF232F6E
:1011A000291B482F249F020E20E0211D1124321BF1
:1011B000232FD1CF1F93DC01FB017C9111964C9121
:1011C000119712961C91972F990F990F990F35E54A
:1011D000292F239F020E20E0211D1124822F672F2B
:1011E0006074572F507277FD6FC061115BC0511151
:1011F00005C0922F9095892F90E004C025E5280F17
:1012000090E08BEA4F3F09F424C0442309F47DC0E9
:10121000882331F0382F349F030E30E0311D832FA7
:10122000222321F0249F020E20E0211D992331F07A
:10123000392F349F030E30E0311D932F1124342FAA
:101240003095339F030E30E0311D1124830F230F9F
:10125000930F1F3F09F421C030E0112321F0119FAB
:10126000312D09F03F5F332309F453C0882331F057
:10127000482F439F040E40E0411D842F222321F07C
:10128000239F020E20E0211D992331F0492F439F17
:10129000040E40E0411D942F11248083218392830A
:1012A0001F91089551110BC0392F2AEA329F030E66
:1012B00030E0311D11249BEA931B280F9CCF90E056
:1012C0002095982F80E09ECF611112C051110CC063
:1012D000392F2AEA329F030E30E0311D11242BEA08
:1012E000231B95E5930FEECF922F909520E08ACFA8
:1012F000511106C025E5280F9BEA981B822FF6CFD7
:101300002AEA280F90E0932FF8CF9FEF2FEF8FEF6F
:10131000A0CF90E020E080E0C0CFCF92DF92EF92AC
:10132000FF92CF93CFB7F89480912602882341F1A2
:10133000C0902702D0902802E0902902F0902A0263
:101340000E9454036C197D098E099F096F3F7F43EA
:101350008105910500F1809126028230C8F08091CC
:1013600026028150809326021092050110920401FA
:10137000C092A101D092A201E092A301F092A40137
:1013800080E0CFBFCF91FF90EF90DF90CF90089596
:1013900010922602F5CF81E0F4CF0F931F93CF93E5
:1013A000DF932091A0012F5F322F37703093A0017F
:1013B00020FF2BC020E831FD2064347009F020624A
:1013C000205FFC01EC01239600E011E064856623B8
:1013D00029F070E0C8010E94952A6F5F6187322F63
:1013E000369F030E30E0311D1124311110C01682DA
:1013F000662311F0615061873196EC17FD0731F7D4
:10140000DF91CF911F910F91089520E0D4CF3150FB
:101410003683EECF2F923F924F925F926F927F92E0
:101420008F929F92AF92BF92CF92DF92EF92FF92F4
:101430000F931F93CF93DF9300D000D0CDB7DEB7CB
:101440001C017C836B830E945403D1011F962D9154
:101450003C91621B730B6A307105A8F3F894AB8161
:10146000BC81ED91FC91119758B1546048B14B7F0C
:1014700048B91996CC90199716968C91BC2DB81B2B
:101480008B2FAB81BC8116968C9316971F96BC90C0
:101490001F9712962D913C9113973A8329831C969E
:1014A0006C911C971D967C911D971E96DC901E9743
:1014B0006F5F7F5FD39417969C91179718963C9116
:1014C00018971A96AC901A971B96EC901081A981E8
:1014D000BA8120E0F32E022F322F30811127889419
:1014E0003111380F08F43FEF8195889460FD130F98
:1014F0001795889461FD130F1795889462FD130F5B
:101500001795889463FD130F1795889464FD130F46
:101510001795889465FD130F1795889466FD130F32
:101520001795889467FD130F17958894232F6111E1
:10153000212F8C0D122F002C58B900C0002C17FF42
:1015400048B931812227889400C000C000C000C083
:1015500048B93111390F00C000C0002C58B900C083
:10156000002C16FF48B908F43FEF9195889400C00D
:1015700000C000C000C048B970FD230F00C000C00B
:10158000002C58B900C0002C15FF48B92795889445
:1015900071FD230F00C000C000C000C048B92795EE
:1015A000889400C000C0002C58B900C0002C14FF63
:1015B00048B972FD230F2795889400C000C000C071
:1015C00000C048B973FD230F00C000C0002C58B9FB
:1015D00000C0002C13FF48B92795889474FD230F91
:1015E00000C000C000C000C048B92795889400C062
:1015F00000C0002C58B900C0002C12FF48B975FD7E
:10160000230F2795889400C000C000C000C048B9CF
:1016100076FD230F00C000C0002C58B900C0002C7C
:1016200011FF48B92795889477FD230F00C000C0AB
:1016300000C000C048B92795889400C000C0002CA5
:1016400058B900C0002C10FF48B9132F7111122F88
:101650009A0D00C000C000C000C048B900C000C062
:1016600000C0002C58B900C0002C17FF48B93281C7
:101670002227889400C000C000C000C048B93111C2
:101680003F0D00C000C0002C58B900C0002C16FF50
:1016900048B908F43FEFEB0DF11D00C000C000C0D9
:1016A00000C048B9D0FC230F00C000C0002C58B9BE
:1016B00000C0002C15FF48B927958894D1FC230F52
:1016C00000C000C000C000C048B92795889400C081
:1016D00000C0002C58B900C0002C14FF48B9D2FC3F
:1016E000230F2795889400C000C000C000C048B9EF
:1016F000D3FC230F00C000C0002C58B900C0002C40
:1017000013FF48B927958894D4FC230F00C000C06C
:1017100000C000C048B92795889400C000C0002CC4
:1017200058B900C0002C12FF48B9D5FC230F2795EB
:10173000889400C000C000C000C048B9D6FC230F88
:1017400000C000C0002C58B900C0002C11FF48B9DF
:1017500027958894D7FC230F00C000C000C000C0AC
:1017600048B92795889400C000C0002C58B900C023
:10177000002C10FF48B9132FD110122FF19400C084
:1017800000C000C000C048B9FE0C00C000C000C0CE
:1017900058B900C0002C17FF48B93081222788941F
:1017A00000C000C000C000C048B93111380F00C0EF
:1017B00000C0002C58B900C0002C16FF48B908F42E
:1017C0003FEF8195889400C000C000C000C048B9B8
:1017D00060FD230F00C000C0002C58B900C0002CD1
:1017E00015FF48B92795889461FD230F00C000C0FC
:1017F00000C000C048B92795889400C000C0002CE4
:1018000058B900C0002C14FF48B962FD230F27957A
:10181000889400C000C000C000C048B963FD230F19
:1018200000C000C0002C58B900C0002C13FF48B9FC
:101830002795889464FD230F00C000C000C000C03D
:1018400048B92795889400C000C0002C58B900C042
:10185000002C12FF48B965FD230F2795889400C01E
:1018600000C000C000C048B966FD230F00C000C022
:10187000002C58B900C0002C11FF48B92795889456
:1018800067FD230F00C000C000C000C048B9279505
:10189000889400C000C0002C58B900C0002C10FF74
:1018A00048B9132F6111122F8C0D00C000C000C069
:1018B00000C048B900C0119709F03ECE20E732E0E1
:1018C000A981BA810E94AF2A44E1442E512C612C97
:1018D000712CA30192010E94482A49015A01F12C5E
:1018E000E12CB7018AE9A981BA81A89F0A0E611D7E
:1018F000B89F600D711D11246B0F711D90E080E089
:1019000054E0660F771F881F991F5A95D1F7A301DE
:1019100092010E94162ADA01C901880D991DAA1D9B
:10192000BB1D893EE3E09E07A105B10508F434C064
:10193000885E9340A109B10922E0B695A7959795D5
:1019400087952A95D1F727E0829F080EE11C929F88
:10195000E00CF11C1124E90EF11C20919F0130E0F4
:10196000820F931F8E0D9F1D4091EA015091EB0154
:101970006091EC017091ED01292F3327420F531F25
:10198000611D711D4093EA015093EB016093EC01DE
:101990007093ED0180939F0178940E945403D101CC
:1019A00050967C936E931F970F900F900F900F900F
:1019B000DF91CF911F910F91FF90EF90DF90CF902B
:1019C000BF90AF909F908F907F906F905F904F905F
:1019D0003F902F9008953A9A0895EF92FF920F93B7
:1019E0001F93CF93DF93CDB7DEB762970FB6F8940E
:1019F000DEBF0FBECDBF7C01DC011C968C917A83CB
:101A000069835C834B835E834D830D871E872F879D
:101A1000813001F5CE0101960E94CD0983E0888BCB
:101A20001A8A198AD701ED91FC910484F585E02D7D
:101A3000BE016F5F7F4FC701099562960FB6F8949C
:101A4000DEBF0FBECDBFDF91CF911F910F91FF90F1
:101A5000EF9008951C861B861A86198618861F82A9
:101A6000DDCFEF92FF920F931F93CF93DF93CDB70C
:101A7000DEB762970FB6F894DEBF0FBECDBF7C0114
:101A8000DC011C968C917A8369835C834B835E8333
:101A90004D830D871E872F878130F9F4CE01019683
:101AA0000E94CD09188A1A8A198AD701ED91FC91F2
:101AB0000484F585E02DBE016F5F7F4FC701099556
:101AC00062960FB6F894DEBF0FBECDBFDF91CF9107
:101AD0001F910F91FF90EF9008951C861B861A8628
:101AE000198618861F82DECF80919A0281111AC052
:101AF00090914102809140028F5F2AE0929F800D79
:101B000011248C3360F480932F0280912F026AE0BD
:101B10000E94892A80934102909340020895109276
:101B20002F02F3CF8130B1F49091440280914302AF
:101B30008F5F2AE0929F800D1124883160F480939A
:101B40002E0280912E026AE00E94892A809344022C
:101B500090934302089510922E02F3CF8091520287
:101B6000E2E5F2E09291918392E0E634F907D1F751
:101B700080934602089580914602E6E4F2E0918166
:101B8000919392E0E235F907D1F7809352020895DC
:101B9000ECE3F1E08181819381E0E734F807D1F74C
:101BA0008AE0809347010895E6E4F2E01082118212
:101BB000128281E0838314821582168287831086C5
:101BC000118612868387148608950F931F93CF93EF
:101BD000DF9300D01F92CDB7DEB71092B6030CE6AC
:101BE00012E019821A821B82B801CE0101960E946E
:101BF000DA080D5F1F4F82E00E37180791F70E9439
:101C000056050F900F900F90DF91CF911F910F917C
:101C10000895ECE3F1E080912C02858380910A0124
:101C2000848380910D01838380912D028283809132
:101C30000B01818380910C018083089530914402CF
:101C400030930C019091430290930B01409141021B
:101C500040932D028091400280930D0110920A0161
:101C600010922C0210929F0210925502109256026E
:101C700010925702109258022AE0429F800D1124C0
:101C800080932F02329F900D112490932E02ECEC42
:101C9000F2E09283818310820E9470070C94090EF7
:101CA00090E080E00895FC018585968508950F9366
:101CB0001F93CF93DF9300D01F92CDB7DEB7AB0158
:101CC00019821A821B82DC01ED91FC910190F08156
:101CD000E02D00E010E020E0BE016F5F7F4F09952E
:101CE0000F900F900F90DF91CF911F910F9108955A
:101CF0008F929F92AF92BF92CF92DF92EF92FF921C
:101D00008091040190910501892B71F10E94540387
:101D10004B015C018091270290912802A091290239
:101D2000B0912A0275016401C81AD90AEA0AFB0AAD
:101D30008092270290922802A0922902B0922A0251
:101D4000C114D10481E0E806F10428F48FEFC8162D
:101D50008FE3D80640F18091260281110EC0809158
:101D600026028F5F80932602FF90EF90DF90CF9046
:101D7000BF90AF909F908F90089580912602813000
:101D800099F38091260281508093260210920501DA
:101D9000109204018092A1019092A201A092A3014D
:101DA000B092A401E1CF809126028823E9F28091CC
:101DB00026028230B0F12091040130910501C90161
:101DC000880F991F820F931F9695879596958795F3
:101DD000E0E0C816D90670F0C601880F991F8C0D77
:101DE0009D1D9695879596958795E2E0281739076A
:101DF00008F0E1E0209106013091070140910801CF
:101E00005091090163E971E080E091E00E94792A34
:101E10006E276093060170930701809308019093E9
:101E20000901809126028F5F80932602809126020D
:101E30008F3F09F4ABCFD0920501C092040194CF3B
:101E4000CF92DF92EF92FF9280919A02811147C068
:101E50000E94DA03C0903A02D0903B02E0903C022C
:101E6000F0903D026C197D098E099F09633371055D
:101E70008105910528F08AE080934001809341011B
:101E80000E94DA036C197D098E099F096536710578
:101E90008105910590F00E94DA0360933A027093F5
:101EA0003B0280933C0290933D0280913F028093DD
:101EB000400180913E0280934101809144028093D1
:101EC0003C018091430280933D018AE080933E0172
:101ED00080933F01FF90EF90DF90CF900895909115
:101EE0003F029093400190913E02909341018130D6
:101EF00021F70E94DA03C0903A02D0903B02E090B2
:101F00003C02F0903D026C197D098E099F096333F4
:101F100071058105910528F08AE080933C0180934A
:101F20003D010E94DA036C197D098E099F0965360F
:101F300071058105910548F20E94DA0360933A0227
:101F400070933B0280933C0290933D02B6CFCF92B8
:101F5000DF92EF92FF9280919A02811147C00E9416
:101F6000DA03C0903A02D0903B02E0903C02F0903D
:101F70003D026C197D098E099F0963337105810546
:101F8000910528F08AE080933E0180933F010E94F2
:101F9000DA036C197D098E099F0965367105810583
:101FA000910590F00E94DA0360933A0270933B022D
:101FB00080933C0290933D028091410280933E01C8
:101FC0008091400280933F018091440280933C01C4
:101FD0008091430280933D018AE080934001809389
:101FE0004101FF90EF90DF90CF90089590914102D2
:101FF00090933E019091400290933F01813021F7F0
:102000000E94DA03C0903A02D0903B02E0903C027A
:10201000F0903D026C197D098E099F0963337105AB
:102020008105910528F08AE080933C0180933D0171
:102030000E94DA036C197D098E099F0965367105C6
:102040008105910548F20E94DA0360933A02709389
:102050003B0280933C0290933D02B6CF8A3008F059
:1020600056C0E82FF0E0E95CFF4E0C94A92A41101D
:102070004710551065106B106D106F1071107310B4
:102080007D1060E089E00E94D20260E013C060E051
:1020900089E00E94D20260E08AE00E94D20260E001
:1020A0008BE00E94D20261E00DC060E089E00E94F6
:1020B000D20261E08AE00E94D20260E08BE00E94DE
:1020C000D20260E08CE00C94D20260E089E00E94D1
:1020D000D20261E0E1CF61E0D5CF61E0D9CF61E02C
:1020E000E5CF61E0F3CF60E089E00E94D20260E0DA
:1020F0008AE00E94D20261E0E1CF60E089E00E94C4
:10210000D20260E08AE00E94D20261E0C9CF61E0C1
:1021100089E00E94D20261E0F5CFCF93DF9381E0A6
:102120008093F70288E6809318031092CB031092F5
:10213000CA0360E08EEC93E00E94410781E00E94B8
:102140001301882321F080E0DF91CF9108959091D1
:10215000C9039111FCCF91E09093C9039093C803F8
:102160002FEF2093F6021092F50226E02093F4025E
:102170009093D3029091D302906D9093D30290915B
:10218000C703913009F08AC01092C7039091D3021F
:102190009093BB009091BC0093FDF8CF95EC909389
:1021A000BC009091C9039130E1F39091F502973012
:1021B00008F076C09091F502A4EDB2E0ECEAF2E00E
:1021C000891370C01092CD038093CC03873008F43C
:1021D000BACF8EEC93E00E940107C82F982F9295FA
:1021E0009770DAE08C2F8F709D9F800D1124809363
:1021F000CC028EEC93E00E940107982F92959F707D
:102200008F709D9F800D11248093CD028EEC93E002
:102210000E940107982F929593708F709D9F800D5B
:1022200011248093CE028EEC93E00E940107982F38
:1022300092959F708F709D9F800D11248093CF0287
:102240008EEC93E00E940107982F92959F708F70FB
:102250009D9F800D11248093D0028EEC93E00E940C
:102260000107982F92959F708F709D9F800D11246C
:102270008093D1028EEC93E00E940107982F9295F3
:102280009F708F70825E9D9F800D11248093D2027B
:102290008C2F8095881F8827881F56CF95EE7FCF7B
:1022A00097E08ACF2D9121938F5F8ACF0E948D1066
:1022B000ECECF2E082812AE0622F0E94892A80936E
:1022C0000C0190930B0181810E94892A80932D0239
:1022D00090930D0180810E94892A80930A01909336
:1022E0002C020C94090E80919402882371F01092B4
:1022F0008F0210928E020E94510560918E027091A1
:102300008F028DE090E00C94012A1092530280918C
:102310000C018093440280910B01809343028091D1
:102320002D028093410280910D0180934002109212
:102330003F0210923E0281E080939F020E94DA03E6
:1023400060933A0270933B0280933C0290933D026B
:102350001092550210925602109257021092580293
:1023600062E073E08FE00C94F7040E94CA2A1F9287
:102370000F920FB60F9211242F933F934F935F93B9
:102380006F937F938F939F93AF93BF93EF93FF933D
:1023900089E193E00E94F801FF91EF91BF91AF9125
:1023A0009F918F917F916F915F914F913F912F916D
:1023B0000F900FBE0F901F9018951F920F920FB69F
:1023C0000F9211242F938F939F93EF93FF93E0919C
:1023D0002903F0912A038081E0912F03F0913003CB
:1023E00082FD1BC09081809132038F5F8F7320919B
:1023F0003303821741F0E0913203F0E0E75EFC4FD7
:10240000958F80933203FF91EF919F918F912F9140
:102410000F900FBE0F901F9018958081F4CF1F92E0
:102420000F920FB60F9211244F935F936F937F9388
:102430008F939F934091EA015091EB016091EC01E1
:102440007091ED018091E9019091E801943019F5C6
:102450001092E8019091E80190FD21C08A598D37D2
:1024600028F08D574F5F5F4F6F4F7F4F8093E9018B
:102470004093EA015093EB016093EC017093ED01FE
:102480009F918F917F916F915F914F910F900FBEB0
:102490000F901F9018959F5F9093E801DBCF8959AB
:1024A000DECF1F920F920FB60F9211242F933F93FE
:1024B0004F935F936F937F938F939F93AF93BF934C
:1024C000EF93FF93E0910201F09103010995FF91D1
:1024D000EF91BF91AF919F918F917F916F915F919C
:1024E0004F913F912F910F900FBE0F901F90189515
:1024F0001F920F920FB60F9211242F933F934F9379
:102500005F936F937F938F939F93AF93BF93EF935B
:10251000FF93E0910001F09101010995FF91EF9186
:10252000BF91AF919F918F917F916F915F914F91EB
:102530003F912F910F900FBE0F901F9018951F92F3
:102540000F920FB60F9211242F933F934F935F93E7
:102550006F937F938F939F93AF93BF93EF93FF936B
:102560008091B900887F803609F44AC0F0F588323E
:1025700009F4A7C018F5803109F49BC0B8F488238A
:1025800009F4F9C0883009F494C0FF91EF91BF912C
:10259000AF919F918F917F916F915F914F913F91FB
:1025A0002F910F900FBE0F901F901895883109F44E
:1025B00088C0803251F78093F60214C0803409F449
:1025C0009DC040F48033B9F38833F9F68093F60266
:1025D00085ECB0C0803509F485C0883509F496C013
:1025E000883499F60E94C006D0CF883909F48CC08F
:1025F00038F5883729F050F4883611F0803729F6FD
:1026000083E08093C9031092E70157C0883809F42A
:102610007BC0803919F0803809F0B7CF8091E7018D
:10262000803208F071C0E091E70181E08E0F809365
:10263000E7018091BB00F0E0E953FE4F80833DC08D
:10264000803B39F0E0F4803A09F479C0883A09F027
:102650009CCF84E08093C9031092C6011092C501FB
:10266000E091C503F091C60309958091C5018111E0
:102670000FC081E08093C5011092A50109C0803C84
:1026800009F4A6CF883C09F4A3CF883B09F07DCF9D
:10269000E091C60181E08E0F8093C601F0E0EB551A
:1026A000FE4F80818093BB009091C6018091C5014F
:1026B00029C08091D3028093BB0085EC8093BC003D
:1026C00064CF9091F5028091F402981758F5E0914B
:1026D000F50281E08E0F8093F502F0E0EC52FD4FA1
:1026E0008081E9CFE091F50281E08E0F8093F502C1
:1026F0008091BB00F0E0EC52FD4F80839091F50299
:102700008091F4029817C8F285E8D8CFE091F502DD
:1027100081E08E0F8093F5028091BB00F0E0EC52D7
:10272000FD4F80838091C80381115CCF81E080934D
:10273000C70384EA8093BC001092C90326CF85ECBE
:102740008093BC001092C9038091E701803230F47D
:10275000E091E701F0E0E953FE4F10826091E7015C
:1027600070E0E091C303F091C40387EC91E0099518
:102770001092E7010ACF1092F60234CF1F920F9207
:102780000FB60F9211242F933F934F935F936F9344
:102790007F938F939F93AF93BF93CF93EF93FF93C9
:1027A00080919E01823009F47EC0F8F48823E1F123
:1027B000813009F45CC080919E018F5F863008F003
:1027C000CBC080939E01FF91EF91CF91BF91AF91CC
:1027D0009F918F917F916F915F914F913F912F9139
:1027E0000F900FBE0F901F901895843009F493C07E
:1027F00008F475C08530F9F6C0914101CA3008F07F
:10280000A6C061E085E00E94D2028C2F0E942E10AB
:102810008091500261E0813009F060E081E10E9426
:10282000D2028091510216C0C0913C01CA30D0F44E
:1028300061E088E00E94D2028C2F0E942E108091CD
:10284000460261E0813009F060E081E10E94D2023D
:102850008091470261E0813009F060E087E00E94EA
:10286000D202A9CF60E088E00E94D202E8CFC091F6
:102870003D01CA3098F461E08EE00E94D2028C2FB4
:102880000E942E108091480261E0813009F060E0E2
:1028900081E10E94D20280914902DCCF60E08EE0AB
:1028A0000E94D202EFCFC0913E01CA3098F461E09D
:1028B0008FE00E94D2028C2F0E942E1080914A023B
:1028C00061E0813009F060E081E10E94D2028091F4
:1028D0004B02C0CF60E08FE00E94D202EFCFC091E8
:1028E0003F01CA3098F461E084E00E94D2028C2F4C
:1028F0000E942E1080914C0261E0813009F060E06E
:1029000081E10E94D20280914D02A4CF60E084E078
:102910000E94D202EFCFC0914001CA3098F461E02A
:1029200083E00E94D2028C2F0E942E1080914E02D2
:1029300061E0813009F060E081E10E94D202809183
:102940004F0288CF60E083E00E94D202EFCF60E0C8
:1029500085E00E94D2025CCF10929E0134CF1F927C
:102960000F920FB60F9211242F933F934F935F93C3
:102970006F937F938F939F93AF93BF93EF93FF9347
:1029800060E088E00E94D20260E08EE00E94D20205
:1029900060E08FE00E94D20260E084E00E94D202F8
:1029A00060E083E00E94D20260E085E00E94D202F3
:1029B0008AE00E942E10FF91EF91BF91AF919F91FD
:1029C0008F917F916F915F914F913F912F910F90D8
:1029D0000FBE0F901F901895CF93DF93E9E1F3E0BE
:1029E0001382128288EE93E0A0E0B0E084839583A6
:1029F000A683B7832EE731E03183208325EC30E0D6
:102A00003587248724EC30E03787268720EC30E0B8
:102A1000318B208B21EC30E0338B228B22EC30E0A9
:102A2000358B248B26EC30E0378B268B118E128E63
:102A3000138E148EEEECF3E013821282848395835E
:102A4000A683B78380E991E091838083E6EBF3E08E
:102A50008FEF808312821182148613868FEF9FEF8F
:102A6000DC0187839087A187B2871092CD031092F3
:102A7000CC031092CB031092CA031092C90381E0D9
:102A80008093C8031092C70361E082E10E94D202E2
:102A900061E083E10E94D202E9EBF0E080818E7F69
:102AA000808380818D7F80838CE58093B80085E46E
:102AB0008093BC0081E191E09093C6038093C503AD
:102AC00082E191E09093C4038093C303CAEDD3E005
:102AD00084EF91E0A0E0B0E08E839F83A887B98760
:102AE0008AE0EEE4F1E0AEEEB3E001900D928A955B
:102AF000E1F71E8E82E08F8F1CA21DA2DF91CF9185
:102B00000895CF93DF9300D01F92CDB7DEB77894AE
:102B100084B5836084BD85B5836085BD80916E007A
:102B2000816080936E0082E08093810080918100BB
:102B3000816080938100809180008160809380001B
:102B40008091B10084608093B1008091B000816079
:102B50008093B00087E880937A001092C1008FE0E4
:102B60000E943C03BC01990F880B990B61157105FC
:102B70008105910511F00E94DC2982E090E00E941D
:102B8000E52991E0811101C090E09093360284E044
:102B900090E00E94E529082F8093100183E090E0E7
:102BA0000E94E529182F8093340281E090E00E9472
:102BB000E52980933502083110F010921001183188
:102BC00010F010921001853010F0109235028091B3
:102BD0001001181308C0109234021092360210929D
:102BE0003502109253028BE090E00E94E529082FF5
:102BF000809345028AE090E00E94E529182F809397
:102C0000420280E090E00E94E52991E0811101C03C
:102C100090E090932B02083110F0109245021C3383
:102C200010F01092420289E090E00E94E529182FEE
:102C30008093370288E090E00E94E5298093380273
:102C40001C3310F010923702883110F010923802C5
:102C500087E090E00E94E529082F8093120186E02A
:102C600090E00E94E529182F8093110185E090E003
:102C70000E94E52991E0811101C090E09093320219
:102C8000083110F010921201183110F01092110159
:102C90009091110180911201981302C0109232029A
:102CA0008CE090E00E94E52991E0811101C090E064
:102CB000909333028DE090E00E94ED2990938F0273
:102CC00080938E02853F914020F010928F021092E7
:102CD0008E0261E08CE00E94000361E08BE00E94C4
:102CE000000361E08AE00E94000361E089E00E9445
:102CF000000361E081E10E94000361E087E00E943F
:102D0000000361E088E00E94000361E08EE00E9421
:102D1000000361E08FE00E94000361E084E00E9414
:102D2000000361E083E00E94000361E085E00E940F
:102D3000000361E082E00E94000360E086E00E9400
:102D4000000360E086E00E94D20260E08DE00E9415
:102D5000000360E08DE00E94D20260E086E00E9405
:102D6000000360E086E00E94D20260E087E00E94FB
:102D7000000360E087E00E94D202E0912903F09115
:102D80002A0382E08083E0912503F091260311E07D
:102D90001083E0912703F091280383E08083109251
:102DA0003103E0912D03F0912E0386E08083E091C2
:102DB0002B03F0912C03808188698083E0912B03A1
:102DC000F0912C0380818F7D808389E193E0909343
:102DD000DB038093DA031093F20370E060E08CE091
:102DE0000E94F70460ED77E080E090E00E946806C2
:102DF00068EC70E080E090E00E94A7031092FE0370
:102E000080910102811144C01092F3011092F201ED
:102E10008FEF8093F6018093F7018093F801809300
:102E2000F9018093FA018093FB011093FC01109249
:102E3000FE011092FD011092F5011092F4018091B3
:102E4000A6029091A702892B31F480EF91E0909334
:102E5000A7028093A602E091EE01F091EF01309776
:102E600021F080EF91E09583848380EF91E090934F
:102E7000EF018093EE01109200021092FF018CE6A8
:102E800091E09093F1018093F00181E08093010241
:102E90003A9A8CE692E09093F3018093F20186E0F7
:102EA00090E09093FE018093FD018091B903909191
:102EB000BA03A091BB03B091BC03843C39E09307F3
:102EC000A105B10520F484EC99E0A0E0B0E0809386
:102ED000B9039093BA03A093BB03B093BC030E94C1
:102EE000E50D62E082E00E94000388E79EE0909397
:102EF000010180930001809169008C7F8160809343
:102F00006900E89AF8941092800010928100109263
:102F10006F008CED9FEF909389008093880083E091
:102F20008093800099E19093810080936F00789462
:102F3000412C512C32014A9411E023E0822E33E5DA
:102F4000232E32E0332E80914901882351F00E94D4
:102F50008D100E945105109249010E94E50D0E94BA
:102F6000561180919F02811141C20E94DA03C090E4
:102F70001D02D0901E02E0901F02F09020026C19FA
:102F80007D098E099F09693E73408105910508F40A
:102F90003EC10E94DA0360931D0270931E0280936B
:102FA0001F029093200280913302882309F444C0C9
:102FB0000E948D2926E030E040E050E00E94162A71
:102FC000609309020E948D2924E630E040E050E041
:102FD0000E94162A63337105810591056CF1E09119
:102FE0000902F0E0E45CFE4F8AE080830E948D29B4
:102FF00024E630E040E050E00E94162A625E7F4FF7
:103000008F4F9F4F0E94A70380912C028093410114
:1030100080910A018093400180910D0180933F01CE
:1030200080912D0280933E0180910B0180933D01A0
:1030300080910C0180933C0180912C028F5F8093E2
:103040002C0210931C028A3008F4E1C010922C026A
:1030500080910A018F5F80930A0110931B020E94E6
:103060008D1080913602882379F08091530281116E
:103070000BC09091CE0280911001981305C08AE098
:1030800080939F021093530280912B02882349F171
:1030900080915402811125C080918D02811121C03F
:1030A0009091CD028091420298131BC09091CE0264
:1030B00080914502981315C080919402811111C02E
:1030C00061E072E08FE00E94F70410938D020E948D
:1030D000DA0360939002709391028093920290932E
:1030E0009302809139028823A1F09091CD028091C2
:1030F000370298130EC09091CE0280913802981337
:1031000008C080919402882321F0109294020E94BA
:10311000510580910A0190914801992309F47BC3DC
:10312000833099F580912C0281112FC08091190272
:1031300081112BC082E080939F020E94DA0360938A
:1031400095027093960280939702909398020E9442
:103150008D108091CE022AE0622F0E94892A8093EE
:103160000C0190930B018091CD020E94892A8093DB
:103170002D0290930D018091CC020E94892A8093A8
:103180000A0190932C021093190280910A01863053
:10319000F0F110920A0180910D018F5F80930D0173
:1031A00010931A0210925402109219028A3078F188
:1031B00010920D0180912D028F5F80932D0210934C
:1031C0001802863020F110922D0290910B019F5F22
:1031D00090930B011093170280910C01823048F4F8
:1031E0009A3038F010920B018F5F80930C0110938E
:1031F000160280910C01823050F080910B018430D6
:1032000030F010920B0110920C0110931602809175
:103210000E01882309F423C380911C02882319F12D
:10322000809114029091150201969093150280935B
:1032300014028D3D95404CF080913E028F5F80934B
:103240003E02109215021092140280913E02809369
:1032500041018A3040F010923E0210921C0280918F
:103260002C028093410180911B02882319F18091E7
:10327000120290911302019690931302809312020E
:103280008D3D95404CF080913F028F5F80933F02CF
:10329000109213021092120280913F02809340011B
:1032A0008A3040F010923F0210921B0280910A0176
:1032B0008093400180911A02882319F180911002B5
:1032C00090911102019690931102809310028D3D0E
:1032D00095404CF0809140028F5F809340021092A5
:1032E0001102109210028091400280933F018A30B7
:1032F00040F01092400210921A0280910D018093CA
:103300003F0180911802882319F180910E0290915B
:103310000F02019690930F0280930E028D3D95400F
:103320004CF0809141028F5F8093410210920F0216
:1033300010920E028091410280933E018A3040F04B
:10334000109241021092180280912D0280933E014A
:1033500080911702882319F180910C0290910D023F
:10336000019690930D0280930C028D3D95404CF098
:10337000809143028F5F8093430210920D0210925E
:103380000C028091430280933D018A3040F01092FC
:1033900043021092170280910B0180933D018091AE
:1033A0001602882319F180910A0290910B0201966E
:1033B00090930B0280930A028D3D95404CF08091D2
:1033C00044028F5F8093440210920B0210920A0213
:1033D0008091440280933C018A3040F01092440274
:1033E0001092160280910C0180933C0180919F0203
:1033F0008A3009F06CC00E94DA03C0902202D0909B
:103400002302E0902402F09025026C197D098E09B8
:103410009F09643671058105910508F45FC00E941B
:10342000DA03609322027093230280932402909324
:103430002502809121028F5F8A3008F029C2809393
:1034400021028091210280933C0180933D01809371
:103450003E0180933F018093400180934101809120
:1034600036028823D9F10E948D108091CE0290916E
:103470003402891333C010929F02109253022AE043
:10348000622F0E94892A382F492F80930C01909334
:103490000B018091CD020E94892A582FE92F809339
:1034A0002D0290930D018091CC020E94892A809375
:1034B0000A0190932C029093410180934001E09384
:1034C0003F0150933E0140933D0130933C01809178
:1034D0009F02893009F0DFC10E94200F80919F0276
:1034E000863009F06AC20E94A70F00919F0208303F
:1034F00011F40E94A70F809148018823C1F1023086
:10350000B1F50091990200933C0100933D010093B5
:103510003E0100933F0100934001009341010E944E
:10352000DA03C0909502D0909602E0909702F09056
:1035300098026C197D098E099F0964367105810511
:103540009105A8F00E94DA036093950270939602A9
:1035500080939702909398020F5F009399020A302C
:1035600030F00E94090E1092990210929F028091F1
:103570009402882309F444C00E94DA03C0909002A8
:10358000D0909102E0909202F09093026C197D0924
:103590008E099F09643F71408105910588F10E9461
:1035A000DA03609390027093910280939202909359
:1035B00093020E94A5068115924011F586E00E94B3
:1035C000A9020197E9F480918E0290918F020196F1
:1035D000843F41E0940708F0B4C290938F02809337
:1035E0008E0260918E0270918F028DE090E00E94B9
:1035F000012A60918E0270918F0282E10E94F7048D
:1036000080918D02882349F10E94DA03C0909002D4
:10361000D0909102E0909202F09093026C197D0993
:103620008E099F09603D774081059105B0F00E94A9
:10363000DA036093900270939102809392029093C8
:1036400093020E94A5068115924039F486E00E94FB
:10365000A902019711F410928D0280919F0283308C
:1036600009F08BC000918C02043010F50E94DA033F
:10367000C0908802D0908902E0908A02F0908B027C
:103680006C197D098E099F096536710581059105C3
:1036900078F00E94DA036093880270938902809325
:1036A0008A0290938B020E94C80D0F5F00938C02D8
:1036B00000918C028CEF800F823010F50E94DA03AB
:1036C000C0908802D0908902E0908A02F0908B022C
:1036D0006C197D098E099F09653671058105910573
:1036E00078F00E94DA0360938802709389028093D5
:1036F0008A0290938B020E94C80D0F5F00938C0288
:1037000000918C02033011F00C94152980918702EE
:10371000843011F40C94F9280E948D108091D0020D
:103720002AE0622F0E94892A8093420190934301EC
:103730008091D1020E94892A80934401909345018F
:103740008091D20290E08E54984F64E670E00E941F
:10375000952A80938602622F0E94892A80934601CF
:103760009093470180918C02893038F080918702D4
:103770008111EEC184E080939F02809185028430A4
:1037800009F0F5C10E94DA03C0908102D090820254
:10379000E0908302F09084026C197D098E099F09E4
:1037A000643671058105910508F432C20E94DA037E
:1037B00060938102709382028093830290938402CB
:1037C00080917F029091800201968E3F91050CF0CE
:1037D000C7C19093800280937F0282E38093B603F7
:1037E00010927E02FF24FA9400917E02063008F0C7
:1037F000BCC180917F028983FA82FB82089DB0015F
:10380000112464597D4FCE0101960E94DA080F5FA2
:1038100000937E02E9CF833009F0B7CC80912C026F
:103820008111B3CC0E948D108091CE022AE0622FCC
:103830000E94892A80930C0190930B018091CD0204
:103840000E94892A80932D0290930D018091CC02D1
:103850000E94892A80930A0190932C0296CC809131
:103860000C0180933C0180910B0180933D0180917C
:103870002D0280933E0180910D0180933F01809144
:103880000A018093400180912C0280934101AECDCA
:1038900010922102D6CD813009F020CE10929B02E9
:1038A00010929C0210929D0210929E020E94A70FFD
:1038B00085E10E943C0340919B0250919C026091E3
:1038C0009D0270919E0204976CF44F5F5F4F6F4FA3
:1038D0007F4F40939B0250939C0260939D02709394
:1038E0009E02E6CF493E53406105710554F01092A7
:1038F0009B0210929C0210929D0210929E020E94C6
:10390000740D86E00E943C0340919B0250919C0202
:1039100060919D0270919E0204976CF44F5F5F4F1F
:103920006F4F7F4F40939B0250939C0260939D0288
:1039300070939E02E6CF493E5340610571057CF0CD
:1039400010929B0210929C0210929D0210929E0275
:1039500080919A028F5F8230E0F480939A028DE02A
:103960000E94A90240919B0250919C0260919D028D
:1039700070919E02892B81F44F5F5F4F6F4F7F4F95
:1039800040939B0250939C0260939D0270939E0211
:10399000E6CF10929A02E3CF41325E446105710591
:1039A0000CF49CCD10929B0210929C0210929D02EE
:1039B00010929E020E941E0E91CD873019F40E9433
:1039C000200F93CD853009F090CD00919A0201111E
:1039D0006FC00E94DA03C0903A02D0903B02E090A0
:1039E0003C02F0903D026C197D098E099F096333FA
:1039F00071058105910528F08AE08093400180934C
:103A000041010E94DA036C197D098E099F09653610
:103A100071058105910590F00E94DA0360933A02E6
:103A200070933B0280933C0290933D0280913F0251
:103A30008093400180913E02809341018091410238
:103A400080933E018091400280933F01023009F053
:103A50006FC00E94DA03C0903A02D0903B02E0901F
:103A60003C02F0903D026C197D098E099F09633379
:103A700071058105910528F08AE080933C018093CF
:103A80003D010E94DA036C197D098E099F09653694
:103A900071058105910508F428CD0E94DA03609331
:103AA0003A0270933B0280933C0290933D0240C0E7
:103AB00080913F028093400180913E0280934101BA
:103AC000013009F0BBCF0E94DA03C0903A02D090D7
:103AD0003B02E0903C02F0903D026C197D098E099A
:103AE0009F09633371058105910528F08AE0809371
:103AF0003E0180933F010E94DA036C197D098E0913
:103B00009F09653671058105910590F00E94DA03E1
:103B100060933A0270933B0280933C0290933D0283
:103B20008091410280933E018091400280933F0149
:103B30008091440280933C018091430280933D0137
:103B4000D4CC10928F0210928E020E94510549CD62
:103B5000843009F012CE0E94561110929F020DCEB1
:103B60001092800210927F0238CE0E9456058091FA
:103B70008502813009F04CC00E94DA03C0908102B6
:103B8000D0908202E0908302F09084026C197D094B
:103B90008E099F09643671058105910508F47CC082
:103BA0000E94DA0360938102709382028093830201
:103BB0009093840282E38093B60310927E02FF24E6
:103BC000FA9400917E020630A8F4E02FF0E0EC5E5B
:103BD000FE4F80818983FA82FB82089DB001112407
:103BE00064597D4FCE0101960E94DA080F5F009361
:103BF0007E02E7CF0E94560580913B01EBE3F1E0A6
:103C00009291918331E0E431F307D1F7809314016D
:103C100080918502823009F03FC00E94DA03C09093
:103C20008102D0908202E0908302F09084026C19AD
:103C30007D098E099F096A3071058105910508F497
:103C4000AEC00E94DA036093810270938202809377
:103C500083029093840280916B0260911301909192
:103C60006A02891709F4F9C489838FEF8A838AEF7E
:103C70008B83689DB001112464597D4FCE0101965C
:103C80000E94DA0888E78093B6030E945605809167
:103C90006B028F5F80936B0280918502833009F005
:103CA0007EC08EE18093B6030E94DA03C090650265
:103CB000D0906602E0906702F09068026C197D096E
:103CC0008E099F09653171058105910508F467C06A
:103CD0000E94DA0360936502709366028093670224
:103CE000909368029CE6A92E92E0B92ED12CC12CAB
:103CF000E0906302F0906402B701C6010E940F08D1
:103D0000082FB701C6010E940F08982EB701C601FF
:103D10000E940F08282F30E0A5E1B0E00E946A2A37
:103D2000A30192010E94162A205B2983A92DB0E0ED
:103D300026EF3FEF4FEF5FEF0E94352AA30192017C
:103D40000E94162A21503F4F4F4F5F4F2A83202F4A
:103D500030E0A9EBB0E00E946A2AA30192010E9420
:103D6000162A2A5B3F4F4F4F5F4F2B83B501CE0181
:103D700001960E94DA084FE0C40ED11C53E0A50E54
:103D8000B11C8AE5C816D10409F0B2CF94E1E90E5E
:103D9000F11CF0926402E09263020E945605809149
:103DA0006202843009F075C40E94DA03C0905E029A
:103DB000D0905F02E0906002F09061026C197D0982
:103DC0008E099F09653671058105910560F00E9495
:103DD000DA0360935E0270935F02809360029093B7
:103DE00061020E94AE0D8DE00E94A902892B31F480
:103DF00080919F02811102C00E9473110E948D095F
:103E00002FB7F89480910401909105012FBF892B61
:103E100011F00C9401280FB7F8940E948D092FB768
:103E2000F89480910401909105012FBF892B09F02E
:103E300089C40E94540360932702709328028093E0
:103E4000290290932A028091260280910601909186
:103E50000701A0910801B091090125EC3DE94CE171
:103E600051E82093060130930701409308015093D5
:103E700009014FEF5FEF5093050140930401109249
:103E800026020FBF8093550290935602A0935702CB
:103E9000B093580220918D02222399F08D3A964DCD
:103EA000AC41B54171F410928D02109354020E94FE
:103EB000510510925502109256021092570210921C
:103EC00058028091550290915602A0915702B091EC
:103ED00058028D3A964DAC41B541C9F480915302D8
:103EE000882361F010929F021092550210925602A0
:103EF00010925702109258020E945611809194021B
:103F0000882329F070E060E084E00E94F70480914B
:103F1000550290915602A0915702B09158028D3AE5
:103F20009645A44EB84629F51092550210925602B5
:103F300010925702109258028091940290919F0221
:103F4000911133C4811134C4809162028F5F863035
:103F500008F0FCC38093620280916202823009F40F
:103F600007C408F0F6C3882309F4FBC3813009F4C1
:103F7000F5C38091550290915602A0915702B091DD
:103F800058028D3A9647AC47B94271F480919F022E
:103F900081110AC0109255021092560210925702D7
:103FA000109258020E94731180915502909156020E
:103FB000A0915702B09158028D3A934AAB45BE4446
:103FC000C1F580919F02811100C410925502109298
:103FD00056021092570210925802809145022AE030
:103FE000622F0E94892A8093440290934302809119
:103FF00042020E94892A80934102909340021092CB
:104000003F0210923E0286E080939F020E94DA03F4
:1040100060933A0270933B0280933C0290933D027E
:10402000809194028111D1C361E073E08FE00E941E
:10403000F7048091550290915602A0915702B091D9
:1040400058028D3A914EA740B24E09F0BEC38091FE
:104050009F02811138C010925502109256021092A0
:10406000570210925802809139028111A7C38091A2
:1040700038022AE0622F0E94892A8093440290939A
:104080004302809137020E94892A809341029093D3
:10409000400210923F0210923E0288E080939F02FD
:1040A0000E94DA0360933A0270933B0280933C02D1
:1040B00090933D02109339028091940267E073E07F
:1040C000882309F47FC38091550290915602A091F4
:1040D0005702B09158028D3A9846A047B14509F071
:1040E000CAC380919F02811147C01092550210925D
:1040F0005602109257021092580200919402809139
:1041000036028111ADC310939A02109336022091AA
:1041100010013AE0822F632F0E94892A8093440283
:104120009093430230934102309340024091350214
:10413000842F0E94892A80933F0290933E02283167
:1041400018F0453008F08AC3240F283108F02851B0
:104150002093340289E080939F020E94DA036093E7
:104160003A0270933B0280933C0290933D0266E0DA
:1041700073E0002309F47CC38091550290915602AC
:10418000A0915702B09158028D3A9647AC47B94278
:10419000D9F580919F02843009F043C010925502F6
:1041A00010925602109257021092580280913C01D0
:1041B0008093440280913D018093430280913E01AF
:1041C0008093410280913F018093400280914001A1
:1041D00080933F028091410180933E0285E080936D
:1041E0009F020E94DA0360933A0270933B0280932D
:1041F0003C0290933D0280919402811105C064E0DD
:1042000073E08FE00E94F70480915502909156026E
:10421000A0915702B09158028D3A9647AC47B942E7
:1042200071F480919F02813051F4109255021092E6
:10423000560210925702109258020E941E0E809150
:10424000550290915602A0915702B09158028D3AB2
:104250009647AC47B94269F580919F02863049F58F
:1042600010929F021092550210925602109257021D
:1042700010925802209141029AE080914002299FB9
:10428000800D112480934202809144026091430288
:10429000899F600D1124609345028BE090E00E949D
:1042A000F329609142028AE090E00E94F3290E9483
:1042B00056118091550290915602A0915702B091EB
:1042C00058028D3A9647AC47B94279F580919F02E2
:1042D000883059F510929F021092550210925602A2
:1042E00010925702109258021093390280914102A5
:1042F0009AE060914002899F600D1124609337021B
:104300002091440280914302299F800D11248093C3
:10431000380289E090E00E94F3296091380288E039
:1043200090E00E94F3290E945611809155029091CD
:104330005602A0915702B09158028D3A9647AC4769
:10434000B942B9F580919F02873099F510929F028A
:104350001092550210925602109257021092580273
:1043600020913F029AE080913E02299F800D112406
:10437000809311012091440260914302299F600DB6
:104380001124609312018613AAC21092320287E0B0
:1043900090E00E94F3296091110186E090E00E9474
:1043A000F3296091320285E090E00E94F3290E9497
:1043B00056118091550290915602A0915702B091EA
:1043C00058028D3A9647AC47B94209F04CC08091EB
:1043D0009F02893009F047C010929F021092550247
:1043E0001092560210925702109258028091440285
:1043F0009AE060914302899F600D1124609310013F
:1044000020913F0280913E02299F800D11248093CC
:104410003502683118F09EE1853028F4962F980F08
:10442000983108F098519093340281115BC2109238
:1044300036021092530284E090E00E94F3296091CA
:10444000340283E090E00E94F3296091360282E01A
:1044500090E00E94F3296091350281E090E00E9493
:10446000F3290E9456118091550290915602A09115
:104470005702B09158028D3A9647AC47B94289F538
:1044800080919F02853069F5109255021092560274
:104490001092570210925802209144029AE08091A3
:1044A0004302299F800D11248093D0022091410264
:1044B00080914002299F800D11248093D102209188
:1044C0003F0280913E02299F800D11248093860235
:1044D000825E8093D20210929F020E9470070E9417
:1044E000090E8091550290915602A0915702B09109
:1044F00058028D3A9041A445B24ED9F4109255021B
:1045000010925602109257021092580280919F0208
:10451000813009F4EAC1883009F4E7C1863009F036
:10452000F2C180919A028F5F823008F4FFC110922D
:104530009A028091550290915602A0915702B09133
:1045400058028D3A9445AE4CB441E9F510925502AB
:1045500010925602109257021092580280919F02B8
:1045600081111EC080919402811115C08091850235
:104570008F5F863008F01DC280938502809185028E
:10458000823009F431C208F017C2882309F429C225
:10459000813009F441C28091940281110E94510539
:1045A00080919F02813009F43BC2883009F438C2FF
:1045B000863009F043C280919A028150823008F41B
:1045C00050C210939A028091550290915602A09188
:1045D0005702B09158028D3A9B4EAE49B34F09F045
:1045E00079C2109255021092560210925702109200
:1045F000580280919F02811167C280910F01813022
:1046000009F43FC208F438C2823009F43FC2833053
:1046100009F43FC28AEF8093B60310927E0288E7C6
:10462000E82EFF24FA9400917E02063008F03AC288
:10463000089DF0011124E459FD4F80910F010813EA
:104640002DC2E982FA82FB82BF01CE0101960E944F
:10465000DA080F5F00937E02E6CF90916902909393
:104660006B02662321F061506093130115CB95E036
:10467000909313018093690280936B020E948D29AD
:104680002AEF30E040E050E00E94162A60936A0270
:1046900003CB823099F50E94DA03C0905E02D0907D
:1046A0005F02E0906002F09061026C197D098E0952
:1046B0009F09653671058105910508F494CB0E9428
:1046C000DA0360935E0270935F02809360029093BE
:1046D000610200915D020B3010F40E94BB0D85EF6A
:1046E000800F8B3010F40E94AE0D0F5F063118F46E
:1046F00000935D0278CB10925D0275CB833009F098
:10470000E9C40E94DA03C0905E02D0905F02E0909C
:104710006002F09061026C197D098E099F0965366F
:1047200071058105910508F45ECB0E94DA03609360
:104730005E0270935F0280936002909361020E9418
:10474000BB0D51CB80E090E0DC019BCB109262026C
:1047500003CC853078F0853009F00BCC0E94D40D65
:1047600008CCE6E4F2E011922E163F06E1F701CC08
:1047700010925D0210924602109247021092480277
:104780001092490210924A0210924B0210924C026F
:1047900010924D0210924E0210924F02109250024F
:1047A0001093510210925202E4CB882309F4E1CB1A
:1047B00070E060E085E00E94F704DBCB10923902E4
:1047C00068E073E08FE00E94F704809155029091B9
:1047D0005602A0915702B09158028D3A964AAC41C8
:1047E000B54E09F070CC80919F02811144C01092A7
:1047F00055021092560210925702109258021093CE
:104800009A02809112012AE0622F0E94892A8093E5
:1048100044029093430220934102209340028091EE
:1048200011010E94892A80933F0290933E0287E003
:1048300080939F020E94DA0360933A0270933B02D6
:1048400080933C0290933D0280919402811113C0A9
:1048500065E073E08FE00E94F70435CC2EE178CC60
:104860001092360210925302011186CC6BE073E075
:104870008FE00E94F7048091550290915602A0911A
:104880005702B09158028D3A9D4DA249BB4109F0A3
:1048900073CC80919F0281116FCC109255021092BF
:1048A00056021092570210925802809133028111E1
:1048B0000EC069E073E08FE00E94F70410933302AA
:1048C000609133028CE090E00E94F32955CC6AE0BD
:1048D00073E08FE00E94F70410923302F1CF10933F
:1048E000320255CD10933602A6CD90919A029F5F69
:1048F000923018F490939A0211CE10929A02863058
:1049000011F481E013C0873011F0893039F49091AF
:104910009A029F5F923068F490939A02853081F4F6
:1049200080919A028F5F833008F001CE80939A02C3
:1049300000CE853019F410939A02FBCD10929A02A2
:104940008111F7CD809194028823B1F080918E027D
:1049500090918F028230910538F1029790938F02E7
:1049600080938E0260918E0270918F028DE090E0B4
:104970000E94012A0E945105809194028111D9CD93
:104980000E94DA03609390027093910280939202E6
:10499000909393021093940260918E0270918F0213
:1049A00082E10E94F704C5CD10928F0210928E0210
:1049B000D9CF10928502E2CD843071F108F0EBCDB1
:1049C00082E38093B60333E0309385020E94DA03DA
:1049D0006093810270938202809383029093840299
:1049E000DACD0E94E50DD7CD82E38093B6030E9415
:1049F000DA03609381027093820280938302909322
:104A000084020E948D292AEF30E040E050E00E94AD
:104A1000162A60936902BFCD82E38093B603D6CF96
:104A200090919A029150923018F490939A02C0CDCE
:104A300010939A02863011F480E013C0873011F091
:104A4000893039F490919A029150923068F49093A1
:104A50009A02853009F0B7CD80919A028150833057
:104A600048F480939A02AFCD10939A02853009F0F2
:104A7000AACDE2CF82E0F5CF10920E01109248014C
:104A8000C9CD10920E0180934801C4CD10930E0140
:104A9000F5CF10930E0110934801BCCD1082118206
:104AA0001282D7CD0E94560564E670E080E090E067
:104AB0000E94A7030E94E50D80910F018F5F843053
:104AC00008F03FC080930F0180919F028130E1F593
:104AD0000E94740D8091550290915602A091570248
:104AE000B09158028D3A964FA948B04C09F022C2B5
:104AF00010925502109256021092570210925802CC
:104B000080919F02813009F038C180919A02811111
:104B100018C1909141028091400281502AE0929FF9
:104B2000800D11248C3308F00AC180932F028091EC
:104B30002F026AE00E94892A8093410290934002EA
:104B400090C110920F01C0CF8630D9F580919A02A2
:104B500081111AC0809140028F5F909141025AE00A
:104B6000959F800D11248C3360F4809342028091D4
:104B700042026AE00E94892A809341029093400297
:104B8000A9CF10924202F3CF813009F0A3CF9091C8
:104B90004402809143028F5F2AE0929F800D11248E
:104BA000883160F480934502809145026AE00E945A
:104BB000892A80934402909343028CCF109245023D
:104BC000F3CF883009F0D1C280919A02811113C0CD
:104BD00090914102809140028F5F3AE0939F800D57
:104BE00011248C3328F48093370280913702C1CF8F
:104BF00010923702FACF813009F06CCF80914302D6
:104C00008F5F909144024AE0949F800D1124883177
:104C100028F48093380280913802C8CF109238026D
:104C2000FACF80919A0281111AC090913F0280912F
:104C30003E028F5F5AE0959F800D1124883160F409
:104C400080931101809111016AE00E94892A80936A
:104C50003F0290933E023ECF10921101F3CF81307C
:104C600009F038CF90914402809143028F5F2AE08F
:104C7000929F800D1124883128F480931201809135
:104C8000120194CF10921201FACF80919A028111F1
:104C900013C090913F0280913E028F5F3AE0939F54
:104CA000800D1124853028F48093340280913402E1
:104CB000CBCF10923402FACF813009F00BCF909114
:104CC0004402809143028F5F4AE0949F800D11243B
:104CD000883128F4809310018091100167CF1092E1
:104CE0001001FACF84E15AC2913099F42091410227
:104CF000809140028F5F3AE0239F800D11248D3018
:104D000028F4809331028091310233CF90933102A5
:104D1000FACF923009F0DECE809143028F5F9091FE
:104D200044024AE0949F800D1124803228F480933D
:104D30003002809130023ACF10933002FACF8BE3E9
:104D4000F4CE813009F08DC09091440280914302ED
:104D500081503AE0939F800D1124883160F4809354
:104D60002E0280912E026AE00E94892A80934402DA
:104D70009093430276C087E1F2CF863059F5809157
:104D80009A02811112C0909141028091400281509B
:104D90004AE0949F800D11248C3328F480934202C2
:104DA00080914202C6CE8BE3F9CF813009F059C021
:104DB000909144028091430281505AE0959F800D6A
:104DC0001124883128F48093450280914502CBCF8D
:104DD00087E1F9CF883009F0E6C180919A0281110C
:104DE00012C0909141028091400281502AE0929F2E
:104DF000800D11248C3328F4809337028091370280
:104E000098CE8BE3F9CF813061F590914402809187
:104E1000430281503AE0939F800D1124883128F499
:104E200080933802809138029ECF87E1F9CF80913C
:104E30009A0281113CC090913F0280913E028150C4
:104E40004AE0949F800D1124883178F580931101F8
:104E5000809111016AE00E94892A80933F02909319
:104E60003E0200919F02043009F064C010928C024F
:104E70000E94DA03609388027093890280938A0209
:104E800090938B020093870243E040939F028AE055
:104E900080934201809343018093440180934501B4
:104EA000809346018093470145C087E1CFCF813091
:104EB000C1F6909144028091430281505AE0959F3F
:104EC000800D1124883128F4809312018091120101
:104ED0004ACF87E1F9CF80919A02811112C0909157
:104EE0003F0280913E0281502AE0929F800D112462
:104EF000853028F48093340280913402ABCF84E073
:104F0000F9CF8130B9F490914402809143028150ED
:104F10003AE0939F800D1124883108F082C080937D
:104F20001001809110016AE00E94892A8093440256
:104F3000909343028091550290915602A09157029E
:104F4000B09158028D3A9642AA48B04F89F58091A7
:104F50009F0281112DC0109255021092560210929C
:104F60005702109258028091940281119BC0909137
:104F70002D022AE080910D01929F800D11248093D3
:104F80002F0230910C0190910B01329F900D112452
:104F900090932E029093CE028093CD021092CC0279
:104FA0000E94700710920A0110922C020E94090EB2
:104FB0008091550290915602A0915702B0915802EB
:104FC0008D3A9645AA42BC4AA1F41092550210921D
:104FD0005602109257021092580280912B02882399
:104FE00009F473C010922B026DE073E08FE00E9411
:104FF000F704109255021092560210925702109226
:10500000580240E050E0452B11F40C94A3170E9485
:10501000E401882311F40C949C170E9400000C9466
:105020009C1787E17CCF80919A02811112C09091E8
:105030003F0280913E0281504AE0949F800D1124EE
:10504000843128F0809386028091860203CF8CE31E
:10505000F9CF813091F490914102809140028150CA
:105060005AE0959F800D1124882329F08093310206
:10507000809131025ECD8CE0F9CF823009F0F1CE23
:10508000909144028091430281502AE0929F800DCA
:105090001124882329F0809330028091300263CE5E
:1050A0008FE1F9CF109294020E94510560918E0217
:1050B00070918F026150710970938F0260938E021C
:1050C0008DE090E00E94012A73CF10932B026CE0D8
:1050D00073E08CCF853011F00C94F31E0E94DA033C
:1050E000C0905E02D0905F02E0906002F09061029A
:1050F0009B01AC012C193D094E095F0969017A0138
:10510000C0925902D0925A02E0925B02F0925C0285
:1051100035E6C316D104E104F10434F4E6E4F2E028
:1051200011922E163F06E1F7D701C6018556910967
:10513000A109B10984369105A105B10510F40E94B9
:10514000D40D49ECC416D104E104F10414F40C9418
:10515000F31E0E94DA0360935E0270935F028093F5
:105160006002909361020C94F31E873009F459CDCC
:10517000893009F48ACD853009F0ACCC90919A023F
:105180009111B2CD90913F0280913E028F5F5AE023
:10519000959F800D11248D3308F0A4CD8093860255
:1051A0008091860251CD873009F441CE893009F4CF
:1051B00092CE853009F437CF811153CE10928C02F4
:1051C0000E94DA03609388027093890280938A02B6
:1051D00090938B021092870233E030939F0280916C
:1051E00094028111A7CE63E073E08FE00E94F70480
:1051F00038CE0E948D108091CE022AE0622F0E944C
:10520000892A80934201909343018091CD020E94AC
:10521000892A80934401909345018091CC020E9499
:10522000892A80934601909347018AEF800F83304B
:1052300010F00C94B21B0E94DA03C0908802D09048
:105240008902E0908A02F0908B026C197D098E0928
:105250009F09653671058105910510F40C94B21B08
:105260000E94DA03609388027093890280938A0215
:1052700090938B020E94C80D0F5F00938C020C94D8
:10528000B21B8F929F92AF92BF92CF92DF92EF921A
:10529000FF92CF93DF93EC01688179818A819B81B2
:1052A000611571058105910521F464E279ED8BE5C5
:1052B00097E02DE133EF41E050E00E94162A4901CA
:1052C0005A019B01AC01A7EAB1E40E94352A6B01A7
:1052D0007C01ACEEB4EFA50194010E94432AC60EF6
:1052E000D71EE81EF91EF7FE06C081E0C81AD108D5
:1052F000E10880E8F80AC882D982EA82FB82C70105
:10530000B6019F77DF91CF91FF90EF90DF90CF9024
:10531000BF90AF909F908F9008958F929F92AF9281
:10532000BF92CF92DF92EF92FF9260914A0170910B
:105330004B0180914C0190914D01611571058105E2
:10534000910521F464E279ED8BE597E02DE133EFEF
:1053500041E050E00E94162A49015A019B01AC012C
:10536000A7EAB1E40E94352A6B017C01ACEEB4EFF0
:10537000A50194010E94432AC60ED71EE81EF91EFD
:10538000F7FE06C081E0C81AD108E10880E8F80AF3
:10539000C0924A01D0924B01E0924C01F0924D0133
:1053A000C701B6019F77FF90EF90DF90CF90BF903D
:1053B000AF909F908F90089560934A0170934B0136
:1053C00080934C0190934D010895F999FECF92BDC1
:1053D00081BDF89A992780B50895A8E1B0E042E030
:1053E00050E00C94082A262FF999FECF1FBA92BDDF
:1053F00081BD20BD0FB6F894FA9AF99A0FBE0196B6
:1054000008950E94F329272F0C94F429DC01CB0185
:10541000FC01F999FECF06C0F2BDE1BDF89A3196C4
:1054200000B40D9241505040B8F70895052E97FBF7
:105430001EF400940E942D2A57FD07D00E94482A8E
:1054400007FC03D04EF40C942D2A509540953095CE
:1054500021953F4F4F4F5F4F0895909580957095E0
:1054600061957F4F8F4F9F4F08950E946A2AA59F95
:10547000900DB49F900DA49F800D911D112408954F
:10548000B7FF0C94352A0E94352A821B930B08958E
:10549000A1E21A2EAA1BBB1BFD010DC0AA1FBB1F38
:1054A000EE1FFF1FA217B307E407F50720F0A21BAA
:1054B000B30BE40BF50B661F771F881F991F1A9417
:1054C00069F760957095809590959B01AC01BD0141
:1054D000CF010895A29FB001B39FC001A39F700D9B
:1054E000811D1124911DB29F700D811D1124911DEC
:1054F0000895DB018F939F930E94352ABF91AF914E
:10550000A29F800D911DA39F900DB29F900D11241D
:105510000895991B79E004C0991F961708F0961B0F
:10552000881F7A95C9F78095089597FB072E16F482
:10553000009407D077FD09D00E94B62A07FC05D059
:105540003EF4909581959F4F0895709561957F4F9A
:105550000895EE0FFF1F0590F491E02D09940E942D
:105560006A2AB7FF0895821B930B0895AA1BBB1BE1
:1055700051E107C0AA1FBB1FA617B70710F0A61B53
:10558000B70B881F991F5A95A9F780959095BC0174
:10559000CD01089581E090E0F8940C94CF2AF8941E
:0255A000FFCF3B
:1055A200BF060000FFFFC59D1C8105030209010320
:1055B2000206170500060C12181E242A30363C4239
:1055C200484E545A60666C72787E848A90969CA289
:1055D200A8AEB4BAC0C6CCD2D8DEE4EA000000005D
:1055E20000000A0A0A0A0A0A0101010000007EFFFD
:1055F20006000100000000EF00000000B511B51127
:10560200B511570E530E500E00000000310DED0C77
:10561200EB0C570E530E77010A0A00000000190224
:105622007A01A7016002D801B601CA010000000098
:0E56320041071407FD07F10670010107F2069B
:00000001FF
